:020000040000FA
:0400000023EF00F0FA
:0400080031EF10F0D4
:080018009E928150E76E0D4A33
:1000200004D00E18D8B411000E1A0D50DF6ED92A64
:100030000D6AE12AE950E162110034EC01F0E106B9
:10004000D90602801100D86AF26A9E6AF16AF06AE3
:10005000FA6AFB6A0001D08E026A070EC16E806ADE
:10006000816A826A808AF19E0F0E926EFF0E936EF5
:10007000BF0E946E030E1F6F040E206EA0EC01F0F5
:10008000150E82B8040EAF6E240EAC6E900EAB6EE1
:10009000106A116A126A136A146A156A166A0F6A7C
:1000A0009EBA08D00F2A0FAA808A0FBA809AA0ECB5
:1000B00001F0F6D7AE50046E38EC01F00450490A56
:1000C000D8B4BEEF01F004504A0AD8B4AEEF02F043
:1000D0000450570AD8B4D7EF01F00450580AD8B4E6
:1000E000DDEF01F00450590AD8B4E1EF01F00450FB
:1000F0005A0AD8B4A8EF01F00450440AD8B4B3EFB8
:1001000001F004503F0A27E00450300A72E0045026
:10011000310A73E00450320A74E00450330A75E087
:100120000450340A66E00450350A67E00450360A89
:1001300068E00450370A69E00450380A6AE0045065
:10014000530AD8B47DEF10F00450560AD8B400EF2B
:1001500012F050EF00F0320E38EC01F0360E38ECB1
:1001600001F050EF00F09EAA0AD0AE50390A07E124
:1001700034EC01F0390E38EC01F050EF00F0E150B2
:10018000E95C13E0010EEA6EEF50006E020EEA6EBB
:10019000EF50016EE92A02BAD3EF00F002A26ED846
:1001A00002B285D8E0D7A3D8DED702A0DCD7FE0EF6
:1001B000166E9EAA0AD0AE50390AE1E134EC01F085
:1001C000390E38EC01F050EF00F0010EEA6EEF50FE
:1001D000006E020EEA6EEF50016EE92A02A24ED8BE
:1001E00002B265D8162EE5D7FF0E38EC01F050EFBD
:1001F00000F0130E0C6E18D8B6D7310E0C6E14D852
:10020000B2D7630E0C6E10D8AED7C70E0C6E0CD8DA
:10021000AAD7630E0C6E01D8A6D7808A02900292EC
:10022000028A1A6A1B6A08D0808A0290029A029295
:10023000340E045CD8A8028201EE00F011EE00F04A
:1002400022EE00F00D6A02908150FF0A0E6ECA6A1B
:10025000CC6AF26A9D6A9E6A9F920C50CB6E9D8218
:10026000F28CF28ECA841200CA84F26A809A12005A
:1002700082BAFED79EA8FED7AD6E12000150C00B09
:10028000036E03420340300B8009036E00500F0BD6
:10029000031082BAFED79EA8FED7AD6E01503F0B69
:1002A000400982BAFED79EA8FED7AD6E120001505B
:1002B000C00B036E03420340300B8009036E00380D
:1002C0000C0B031082BAFED79EA8FED7AD6E00506D
:1002D0003F0B82BAFED79EA8FED7AD6E01503F0BF2
:1002E000400982BAFED79EA8FED7AD6E120001501B
:1002F0000DE0400E01600AD001460144036E00503B
:10030000030B1C6E03108DEC01F012001C508DECE1
:1003100001F0400E015EEDE112001A2682BAFED70E
:100320009EA8FED7AD6E1B2A1BA612001A507F0B8B
:1003300082BAFED79EA8FED7AD6E1B6A1A6A12005B
:10034000830E046E056E042EFED7052EFCD7120018
:1003500010EE10F0040E18D8D8A050EF00F0106A7C
:10036000126A50EF00F010EE14F0020E0DD8D8A073
:1003700050EF00F0146A156A50EF00F010EE19F01B
:10038000010E02D850EF00F0808A036E320E0F6E1D
:100390009EBA06D0A0EC01F00F2EFAD7D88012003A
:1003A000AE50E66E65DF032EF1D7D8901200106ACA
:1003B000126A0294029650EF00F00294028650EF07
:1003C00000F00284029650EF00F0165051DF050E47
:1003D0004FDF000E4DDF11EE00F0E65049DFE15037
:1003E000D8B4A0EC01F0060EE262F7D71200D89064
:1003F00002A41200105017E111500AE082A603D0A7
:100400009EAAFCD722D082B612009EAAFCD71DD08D
:1004100082B603D09EAAFCD718D082A628EF02F09D
:100420009EAAFBD712D081501014111803E09EAA87
:10043000FAD70BD01250D8B428EF02F08114131859
:10044000D8B428EF02F09EAAF5D7D880AE5012009B
:1004500014501518D8B4120000001406143C152AC4
:10046000150614501510D8A4F7D7D8901200162AE4
:100470001050D8B4010C11EE00F0050EE26204D069
:100480009EAA000CAE50020C1050E614E652111851
:10049000D8A4F3D71250D8B4010CE7141318D8A479
:1004A000ECD7010C162A1050D8B4010C11EE00F054
:1004B000050EE26204D09EAA000CAE50020C105051
:1004C000E6141118D8A4F4D71250D8B4010CE714CC
:1004D0001318D8A4EDD7010C162A1050D8B4010C6B
:1004E00011EE00F0E7380F0B186E0288050EE2627D
:1004F00004D09EAA000CAE50020C1850176E02A831
:1005000005D00298E6500F0B186E04D00288E73829
:100510000F0B186E105017141118D8A4E7D71250EB
:10052000D8B4010C18141318D8A4E0D7010C00009B
:1005300000000000000000000000000000000000BB
:1005400000000000000000000000000000000000AB
:1005500000000000000000000000010C050EFA6E13
:100560001946194419427C0BF92650EF00F050EF60
:1005700000F043EF04F025EF03F031EF03F031EF2B
:1005800003F050EF00F050EF00F050EF00F09BEF61
:1005900004F01BEF04F00DEF03F019EF03F019EF77
:1005A00003F050EF00F050EF00F0BFEF04F07DEFEC
:1005B00004F0FAEF03F0F5EF02F001EF03F001EFC2
:1005C00003F050EF00F050EF00F050EF00F050EF6C
:1005D00000F050EF00F050EF00F050EF00F050EF5F
:1005E00000F050EF00F050EF00F0808A0290166AA1
:1005F000FEDED8B050EF00F019AE3DEF03F0DAEFB9
:100600000EF0808A0290166AF2DED8B050EF00F049
:1006100019AE3DEF03F07BEF0FF0808A0290166A6F
:10062000E6DED8B050EF00F019AE66EF03F00EEF43
:100630000FF0808A0290166ADADED8B050EF00F030
:1006400019AE66EF03F0B7EF0FF0808A0290166ADA
:10065000CEDED8B050EF00F019AEA5EF03F044EFB6
:100660000FF0808A0290166AC2DED8B050EF00F018
:1006700019AEA5EF03F0F9EF0FF011EE00F081CF06
:10068000E6FF13D8060EE262FAD702A650EF03F097
:1006900052EC02F0010A04E0010AEFE050EF00F032
:1006A000E5EC01F0809A50EF00F01950070B030AB7
:1006B00008E01950070B040A02E0E60E03D0F70E1B
:1006C00001D0FF0E010FFEE100D0120011EE00F08C
:1006D0008138F00BE76E18D881500F0BE710E66EEB
:1006E00024D8060EE262F4D702A67FEF03F06CEC8A
:1006F00002F0010A04E0010AE9E050EF00F0E5EC45
:1007000001F0809A50EF00F01950070B030A08E03F
:100710001950070B040A02E0E50E03D0F60E01D0D3
:10072000FE0E010FFEE100D012001950070B030A64
:1007300008E01950070B040A02E0E60E03D0F70E9A
:1007400001D0FF0E010FFEE1120011EE00F081CF8B
:1007500003F00332E7320332E73228D881CF03F0C7
:100760000332E7320332E73221D881CF03F003327C
:10077000E7320332E7321AD881CF03F00332E7328F
:100780000332E63224D8060EE262E1D702A6D1EFA8
:1007900003F097EC02F0010A04E0010AD6E050EF02
:1007A00000F0E5EC01F0809A50EF00F01950070BD3
:1007B000030A08E01950070B040A02E0E60E03D012
:1007C000F70E01D0FF0E010FFEE100D0120019500C
:1007D000070B030A0AE01950070B040A03E0E70EAF
:1007E000000005D0F80E000002D000001200010F3A
:1007F000FEE11200808A0290166AF9DDD8B050EF4F
:1008000000F011EE00F0060E81CFE6FF000000D0F0
:1008100000D0E262F9D702A616EF04F052EC02F023
:10082000010A04E0010AEDE050EF00F0E5EC01F010
:10083000809A50EF00F0808A0290166AD8DDD8B016
:1008400050EF00F011EE00F08138F00BE76E000081
:1008500000D000D000D081500F0BE710E66E060EDE
:1008600000D0E262F1D702A63EEF04F06CEC02F099
:10087000010A04E0010AE6E050EF00F0E5EC01F0C7
:10088000809A50EF00F0808A0290166AB0DDD8B0EE
:1008900050EF00F011EE00F081CF03F00332E732A9
:1008A0000332E73200D000D081CF03F00332E732C9
:1008B0000332E73200D000D081CF03F00332E732B9
:1008C0000332E73200D000D081CF03F00332E732A9
:1008D0000332E632060EE262DFD702A678EF04F0BA
:1008E00097EC02F0010A04E0010AD4E050EF00F0B6
:1008F000E5EC01F0809A50EF00F0808A0290166AD1
:1009000076DDD8B050EF00F011EE00F0060E81CF8A
:10091000E6FFE262FCD702A696EF04F052EC02F08A
:10092000010A04E0010AF0E050EF00F0E5EC01F00C
:10093000809A50EF00F0808A0290166A58DDD8B095
:1009400050EF00F011EE00F023EE00F08138F00BD4
:10095000E76E0F0EDE528114E612DAA6F7D702A672
:10096000BAEF04F06CEC02F0010A04E0010AEAE0DC
:1009700050EF00F0E5EC01F0809A50EF00F0808A33
:100980000290166A34DDD8B050EF00F011EE00F09E
:1009900081CFE6FF81CFE6FF81CFE6FF81CFE6FF83
:1009A00081CFE6FF81CFE6FF81CFE6FF81CFE6FF73
:1009B00081CFE6FF81CFE6FF81CFE6FF81CFE6FF63
:1009C00081CFE6FF81CFE6FF81CFE6FF81CFE6FF53
:101D900002A6D5EF0EF052EC02F0010A06E0010AAD
:101DA000D8B4C6EF04F050EF00F0E5EC01F0809AF3
:101DB00050EF00F011EE00F081500E6E0D6AE66EED
:101DC000E66A81500D4A1ED00E18D8B420D00E1AE3
:101DD0000E5000D000D0E66E0D50E66E0D6A060E75
:101DE000E262EFD702A6FDEF0EF037EC02F0010A37
:101DF00004E0010ADFE050EF00F0E5EC01F0809A2A
:101E000050EF00F00E6E00D000D00000E4D700D0FC
:101E100000D000D000D000D00000D3D70F0E1D6E30
:101E200011EE00F081501D140E6E0D6AE66E8150A9
:101E30001D140D2A0DB81DD00E18D8B41FD00E1ABF
:101E40000D38F00B0E1000D0E66E0D6A060EE26241
:101E5000EED702A634EF0FF052EC02F0010A04E0D4
:101E6000010ADEE050EF00F0E5EC01F0809A50EF5F
:101E700000F00E6E00D000D00000E6D700D000D0F9
:101E800000D000D00000D3D7030E1D6E11EE00F07D
:101E900081501D140E6E0D6AE66E81501D140D2AC0
:101EA0000DBC1ED00E18D8B420D00E1A0D460D440D
:101EB000FC0B0E100000E66E0D6A060EE262EDD716
:101EC00002A66BEF0FF052EC02F0010A04E0010AE7
:101ED000DDE050EF00F0E5EC01F0809A50EF00F00B
:101EE0000E6E00D000D00000E6D700D000D000D0A9
:101EF00000D00000D2D711EE00F081500E6E0D6AB6
:101F0000E66EE66A81500D4A1DD00E18D8B41DD079
:101F10000E1A21D80E50E66E0D50E66E0D6A060EB2
:101F2000E262F0D702A69DEF0FF037EC02F0010A53
:101F300004E0010AE0E050EF00F0E5EC01F0809AE7
:101F400050EF00F00E6E07D8E5D700D000D000D0DB
:101F5000000001D8D7D71950070B040A03E0E80E98
:101F600000D002D0F80E0000010FFEE112000F0EAB
:101F70001D6E11EE00F081501D140E6E0D6AE66E9E
:101F800081501D140D2A0DB81ED00E18D8B41FD0C4
:101F90000E1A23D80D38F00B0E100000E66E0D6AF5
:101FA000060EE262EDD702A6DEEF0FF052EC02F071
:101FB000010A04E0010ADDE050EF00F0E5EC01F079
:101FC000809A50EF00F00E6EC6DF0E50E7D700D0BB
:101FD00000D000D000D001D8D3D71950070B040A85
:101FE00003E0E90E00D002D0F90E0000010FFEE17F
:101FF0001200030E1D6E11EE00F081501D140E6EC6
:102000000D6AE66E81501D140D2A0DBC1ED00E18EF
:10201000D8B421D00E1AE1DF0D460D44FC0B0E1092
:10202000E66E0D6A060EE262EDD702A620EF10F012
:1020300052EC02F0010A04E0010ADDE050EF00F08A
:10204000E5EC01F0809A50EF00F00E6EC6DF0E5006
:1020500000D00000E5D700D000D000D000D0BDDF18
:10206000D1D79E92811C2C6E346E343232B0213224
:10207000343232B22232343232B42332343232B6D3
:102080002432343232B82532343232BA2632343243
:1020900032BC2732343232BE2832343032142D1260
:1020A0002E502F102C143310356E2C1C2F14321080
:1020B000366E325029142B122D1C3114326E3350CF
:1020C00029122C1C33142A1231502D14336E311C5A
:1020D0002D163050316E2C1C2E142F6E35502E6E56
:1020E0003650306E1F502916110070B8498A70B8EA
:1020F000488A10E608AD00AD0056808A01EE00F077
:1021000011EE00F00290800E216E226E236E246E7E
:10211000256E266E276E286E296A2A6A2D6AFF0EA2
:102120002E6E2F6A306A316A326A336A0F0E1E6E63
:10213000F86A200EF76EEA0EF66E20440E0BF626B5
:10214000CA6ACC6AF26A9D6A9E6A9F820900F5504B
:10215000CA6E0900F550CB6E9D82F28CF28ECA8455
:102160009EAA0AD0AE50390A07E134EC01F0390ECC
:1021700038EC01F050EF00F029B020D829B241D856
:1021800029B462D829B683D829B8A4D829BAC5D821
:1021900029BCE6D829BE07D982BAE2D79EA8E0D7E3
:1021A000E150E95C04E0EF50AD6EE92AD9D702A016
:1021B000D7D7FF0E38EC01F050EF00F02AB00FD067
:1021C0002BB016D0000E1E1804E0000E1E6E800903
:1021D0000DD921500BD92990800E216E12002A9022
:1021E0002990000E1E6EC00901D9800E216E1200CA
:1021F0002B902990000E1E6EA009F8D8800E216E3B
:1022000012002AB20FD02BB216D0010E1E1804E015
:10221000010E1E6E8009EAD82250E8D82992800E5D
:10222000226E12002A922992010E1E6EC009DED87B
:10223000800E226E12002B922992010E1E6EA009B2
:10224000D5D8800E226E12002AB40FD02BB416D02F
:10225000020E1E1804E0020E1E6E8009C7D823501D
:10226000C5D82994800E236E12002A942994020E58
:102270001E6EC009BBD8800E236E12002B942994C9
:10228000020E1E6EA009B2D8800E236E12002AB66E
:102290000FD02BB616D0030E1E1804E0030E1E6ED0
:1022A0008009A4D82450A2D82996800E246E12004A
:1022B0002A962996030E1E6EC00998D8800E246EA9
:1022C00012002B962996030E1E6EA0098FD8800E41
:1022D000246E12002AB80FD02BB816D0040E1E1888
:1022E00004E0040E1E6E800981D825507FD82998FD
:1022F000800E256E12002A982998040E1E6EC009C1
:1023000075D8800E256E12002B982998040E1E6E2B
:10231000A0096CD8800E256E12002ABA0FD02BBAF5
:1023200016D0050E1E1804E0050E1E6E80095ED83C
:1023300026505CD8299A800E266E12002A9A299A75
:10234000050E1E6EC00952D8800E266E12002B9A02
:10235000299A050E1E6EA00949D8800E266E12001D
:102360002ABC0FD02BBC16D0060E1E1804E0060E99
:102370001E6E80093BD8275039D8299C800E276EC5
:1023800012002A9C299C060E1E6EC0092FD8800EB2
:10239000276E12002B9C299C060E1E6EA00926D8C3
:1023A000800E276E12002ABE0FD02BBE16D0070E4D
:1023B0001E1804E0070E1E6E800918D8285016D883
:1023C000299E800E286E12002A9E299E070E1E6EE0
:1023D000C0090CD8800E286E12002B9E299E070E75
:1023E0001E6EA00903D8800E286E1200E76EE12A47
:1023F000E950E162120034EC01F0E10602801200C3
:1024000010EE1FF0020EC4EC01F0D8A050EF00F067
:0C241000030E1F6E040E206E50EF00F053
:020000040030CA
:03000100260E0EBA
:02000500018177
:060008000FC00FE00F40E5
:00000001FF
